:1000000000308A00292800002630840000080319E7
:1000100018280130A100A001A00B0C28A10B0B286F
:100020004A30A000A00B122800000000800B092815
:10003000003494138C11260893000230941B272857
:100040008C1D202800308316111B01308312A10063
:10005000003484011F308305A51525088316870009
:100060008312251625088316870001309300283057
:10007000831294008316941314131F149F141F15D6
:100080009F11FF308312A50083161F149F141F15A4
:100090009F1183121F1083160108C7390838810089
:1000A000831290010030A10092000030831692006C
:1000B0008312251025088316870083120714251341
:1000C00025088316870083120713C830A600042072
:1000D000251025088316870083120710C830A60054
:1000E0000420251025088316870083120714831621
:1000F000111411187928C4308312A6001920123067
:10010000A6001920A430A600192083161115111974
:100110008728111411188A28C4308312A6001920C8
:100120001330A60019200530A600192083161115DA
:1001300011199828FA308312A6000420831611148E
:100140001118A028C4308312A60019203F30A60041
:1001500019204230A6001920831611151119AE2856
:10016000FA308312A6000420251025088316870084
:10017000831207102513250883168700831207179B
:04018000C028630030
:02400E00393F38
:00000001FF
